:100000000C9446000C9463000C9463000C94B103B0
:100010000C94BB030C9463000C9463000C94630079
:100020000C94C5030C9463000C9463000C9463005F
:100030000C94FE030C9463000C9404030C9456037C
:100040000C9463000C9463000C9463000C946300A4
:100050000C9463000C947F030C9463000C94630075
:100060000C9463000C9463000C9463000C94630084
:100070000C9463000C9463000C945B010C9463007B
:100080000C9463000C9463000C94630011241FBE55
:10009000CFEFD0E1DEBFCDBF11E0A0E0B1E0EEE9EF
:1000A000FEE002C005900D92AC32B107D9F721E015
:1000B000ACE2B1E001C01D92A637B207E1F70E94A1
:1000C0009B010C944D070C9400008BBB662331F010
:1000D000E2E6F0E080818460808305C0E2E6F0E043
:1000E00080818B7F8083E2E6F0E08081886080837E
:1000F0008FE19EE40197F1F700C000008081877FC7
:1001000080838FE99FE00197F1F700C00000089518
:10011000CF93C82F60E0807F0E94650060E08C2F45
:100120008295807F0E946500CF9108958FE39CE9BE
:100130000197F1F700C000008FEF8ABBE1E6F0E025
:1001400080818C60808382E00E94880088E20E9427
:1001500088008CE00E94880086E00E94880081E090
:100160000E9488000895CF93C82F61E0807F0E948D
:10017000650061E08C2F8295807F0E946500CF91A1
:1001800008950F931F93CF93DF938C01C0E0D0E0CD
:10019000F801EC0FFD1F8081882321F00E94B3003D
:1001A0002196F6CFDF91CF911F910F910895CF93B4
:1001B000DF93EA01613031F058F0623029F06330AA
:1001C00029F007C090EC05C094E903C094ED01C08C
:1001D00090E88F70892B0E948800CE010E94C10098
:1001E000DF91CF9108951092710088E480937000A0
:1001F00084E080937400089584EA80937400809171
:1002000074008823E4F7089584E980937400809152
:10021000740084FDFCCF089590E0880F991F862B11
:100220008093730084E88093740080917400882325
:10023000E4F780917100887F08958093730084E8CB
:1002400080937400809174008823E4F7809171009A
:10025000887F08959C0140E050E060E271EA87E009
:1002600090E00E94130421503109309398002093AC
:10027000990088E980939A0086E080939D007894A5
:10028000089590919B0095FFFCCF80939C0008956A
:10029000CF93DF93EC018881882321F021960E947F
:1002A0004101F9CF8DE00E9441018AE00E944101A5
:1002B000DF91CF9108951F920F920FB60F921124E4
:1002C0002F933F934F938F939F93AF93BF93EF934E
:1002D000FF934CB1E0E0AE2FB0E0AC5BBE4F8C9131
:1002E000882319F0EF5FE233B1F7E23328F4F0E04E
:1002F000EC5BFE4F408311C020E0213360F4822F7D
:1003000090E0FC01EB5BFE4F3081FC01EC5BFE4FAB
:1003100030832F5FF2CF40937501FF91EF91BF9132
:10032000AF919F918F914F913F912F910F900FBE61
:100330000F901F90189581B3806F81BB9FEF94BB86
:1003400082B3806F82BB97BB8EB583608EBD87B74B
:10035000846087BF1DBC1CBC87B1806487B986B12F
:100360008F6886B986B1806486B9EAE6F0E080815C
:10037000866B80838AB7806C8ABF89B78C6089BF9F
:1003800082B1886382B9EBE8F0E08081886A80837B
:10039000808183608083EAE8F0E0808188608083E8
:1003A000808181608083ECE8F0E08081806E8083D2
:1003B0000E94960080E895E20E942A0141E051E007
:1003C00060E080E00E94D7000E94F3000E94FC00E1
:1003D00060E080E20E940C0181E00E941D010E9409
:1003E00004010E94FC0060E080E20E940C018FEF9B
:1003F0000E941D010E94040182B1846082B9789438
:10040000ECE3F1E022813381808191813F932F934E
:100410009F938F93809143018F93809142018F939B
:1004200081E191E09F938F938CE291E09F938F9372
:100430000E9463044CE251E061E080E00E94D7003A
:100440008CE291E00E9448018DB79EB70A960FB6E4
:10045000F8949EBF0FBE8DBFD3CF80B382958F70AF
:10046000823009F441C018F4813041F0AFC08430CB
:1004700009F467C0883009F48BC0A8C082B38F70BC
:10048000806282BB40914001509141019A013695B2
:1004900027953695279536952795A5ECB0E20E94CD
:1004A0003204929582958F7089279F70892768EE14
:1004B00073E0869F9001879F300D969F300D112429
:1004C000CA01821B930B9C0136952795369527957B
:1004D000ABE7B4E10E94320496958795FC01EF5D8D
:1004E000FE4F808185BB089582B38F70806482BB8C
:1004F00040914001509141019A01369527953695DA
:100500002795ABE7B4E10E9432049C01369527950C
:1005100064E6629FC001639F900D11249A01281B1D
:10052000390BADECBCEC0E943204969587959695FC
:10053000879596958795FC01EF5DFE4F808185BB81
:10054000089582B38F70806882BB409140015091C2
:1005500041019A01ADECBCEC0E943204969587955E
:1005600096958795969587959C01220F331F880F46
:10057000991F880F991F880F991F820F931F9A0147
:10058000281B390BF901EF5DFE4F808185BB089573
:1005900082B38F70806182BB209140013091410114
:1005A000369527953695279536952795A5ECB0E293
:1005B0000E943204929582958F7089279F708927B7
:1005C000FC01EF5DFE4F808185BB089582B38F7083
:1005D000806182BB20914001309141013695279581
:1005E0003695279536952795A5ECB0E20E94320402
:1005F000929582958F7089279F708927FC01EF5D06
:10060000FE4F808185BB08951F920F920FB60F9207
:1006100011242F933F934F935F936F937F938F9307
:100620009F93AF93BF93EF93FF93E0910001E1504D
:10063000E0930001EB3008F187B78B7F87BF89B764
:10064000806889BF1EBC1DBC1CBC88EE93E09BBDAE
:100650008ABD86B7806186BF18BA83B78F6083BFB3
:1006600012BE8AE081BF87B7826087BF8091400158
:10067000909141010E942D0208C0F0E0EF5DFE4F15
:10068000808185BB88B38F5F88BBFF91EF91BF915D
:10069000AF919F918F917F916F915F914F913F911A
:1006A0002F910F900FBE0F901F9018951F920F92D1
:1006B0000FB60F9211242F933F934F935F936F9335
:1006C0007F938F939F93AF93BF93EF93FF9380910B
:1006D0004001909141010E942D0212BEFF91EF91C5
:1006E000BF91AF919F918F917F916F915F914F914A
:1006F0003F912F910F900FBE0F901F9018951F9252
:100700000F920FB60F9211248F939F93389B10C0B6
:1007100084B195B1909383008093820087B18E7FDE
:1007200087B984B195B190933F0180933E010FC08A
:1007300084B195B1909387008093860087B18160E2
:1007400087B984B195B190933D0180933C0186B106
:10075000806486B99F918F910F900FBE0F901F906C
:1007600018951F920F920FB60F9211240F900FBE83
:100770000F901F9018951F920F920FB60F92112491
:100780000F900FBE0F901F9018951F920F920FB6EB
:100790000F9211242F938F939F93809142019091F8
:1007A00043018F3027E2920730F401969093430182
:1007B0008093420104C01092430110924201809143
:1007C000420190914301809340019093410188BB85
:1007D00087B7806187BF8EB588608EBD8EB5856016
:1007E0008EBD1DBC1CBC83B1846083B99F918F9169
:1007F0002F910F900FBE0F901F9018951F920F9280
:100800000FB60F9211248F9387B78F7E87BF83B166
:100810008B7F83B98EB58A7F8EBD8F910F900FBE6F
:100820000F901F901895052E97FB1EF400940E94C0
:100830002A0457FD07D00E94410407FC03D04EF460
:100840000C942A0450954095309521953F4F4F4F79
:100850005F4F089590958095709561957F4F8F4F6C
:100860009F4F0895A29FB001B39FC001A39F700D39
:10087000811D1124911DB29F700D811D1124911DA8
:100880000895A1E21A2EAA1BBB1BFD010DC0AA1FD1
:10089000BB1FEE1FFF1FA217B307E407F50720F0E9
:1008A000A21BB30BE40BF50B661F771F881F991F64
:1008B0001A9469F760957095809590959B01AC01AD
:1008C000BD01CF010895AEE0B0E0E9E6F4E00C949C
:1008D00024070D891E8986E08C831A8309838FEF94
:1008E0009FE79E838D83AE01475E5F4F6F89788D52
:1008F000CE0101960E948504EF81F885E00FF11F7B
:1009000010822E96E4E00C944007ABE0B0E0EBE8F8
:10091000F4E00C9416076C017B018A01FC0117823C
:100920001682838181FFCCC1CE0101963C01F60184
:100930009381F70193FD859193FF81917F01882336
:1009400009F4BAC1853239F493FD859193FF819101
:100950007F01853229F4B60190E00E947C06E7CF42
:10096000912C212C312CFFE1F315D8F08B3279F04A
:1009700038F4803279F08332A1F4232D20611DC038
:100980008D3261F0803369F4232D216016C0832DF0
:100990008260382EE32DE4603E2E2AC0F32DF860ED
:1009A0001DC037FC2DC020ED280F2A3040F08E32BC
:1009B000B9F436FC81C1232D2064322E19C036FED5
:1009C00006C08AE0989E200D1124922E11C0EAE004
:1009D0002E9E200D1124222EF32DF0623F2E08C0F2
:1009E0008C3621F4832D8068382E02C0883641F47D
:1009F000F70193FD859193FF81917F018111B3CF21
:100A0000982F9F7D9554933028F40C5F1F4F9FE3E0
:100A100099830DC0833631F0833771F0833509F047
:100A200059C021C0F801808189830E5F1F4F88243F
:100A30008394912C530113C02801F2E04F0E511CF6
:100A4000F801A080B18036FE03C0692D70E002C0BD
:100A50006FEF7FEFC5010E9471064C018201F32DFB
:100A6000FF773F2E16C0280122E0420E511CF801EC
:100A7000A080B18036FE03C0692D70E002C06FEF28
:100A80007FEFC5010E9466064C01F32DF0683F2EF2
:100A9000820133FC1BC0822D90E088169906B0F4C9
:100AA000B60180E290E00E947C062A94F4CFF50122
:100AB00037FC859137FE81915F01B60190E00E947D
:100AC0007C0621102A9421E0821A91088114910455
:100AD00071F7E8C0843611F0893641F5F80137FE28
:100AE00007C060817181828193810C5F1F4F08C0B4
:100AF00060817181072E000C880B990B0E5F1F4FD0
:100B0000F32DFF763F2E97FF09C090958095709545
:100B100061957F4F8F4F9F4FF0683F2E2AE030E066
:100B2000A3010E94B806882E861845C0853731F487
:100B3000232D2F7EB22E2AE030E025C0932D997F01
:100B4000B92E8F36C1F018F4883579F0B5C08037EA
:100B500019F0883721F0B0C0E92FE061BE2EB4FE55
:100B60000DC0FB2DF460BF2E09C034FE0AC0292F32
:100B70002660B22E06C028E030E005C020E130E05B
:100B800002C020E132E0F801B7FE07C06081718148
:100B9000828193810C5F1F4F06C06081718180E06C
:100BA00090E00E5F1F4FA3010E94B806882E8618A2
:100BB000FB2DFF773F2E36FE0DC0232D2E7FA22E5C
:100BC000891458F434FE0BC032FC09C0832D8E7E8C
:100BD000A82E05C0B82CA32C03C0B82C01C0B92C7A
:100BE000A4FE0FC0FE01E80DF11D8081803321F4C9
:100BF0009A2D997EA92E09C0A2FE06C0B394B39483
:100C000004C08A2D867809F0B394A3FC11C0A0FE1D
:100C100006C0B21488F4280C922C9B180EC0B21493
:100C200060F4B60180E290E00E947C06B394F7CFB6
:100C3000B21418F42B1802C0982C212CA4FE10C05A
:100C4000B60180E390E00E947C06A2FE17C0A1FCE2
:100C500003C088E790E002C088E590E0B6010CC0D0
:100C60008A2D867859F0A1FE02C08BE201C080E295
:100C7000A7FC8DE2B60190E00E947C06891438F44E
:100C8000B60180E390E00E947C069A94F7CF8A94A4
:100C9000F301E80DF11D8081B60190E00E947C0611
:100CA0008110F5CF222009F442CEB60180E290E017
:100CB0000E947C062A94F6CFF6018681978102C0B5
:100CC0008FEF9FEF2B96E2E10C943207FC01059029
:100CD000615070400110D8F7809590958E0F9F1F3E
:100CE0000895FC016150704001900110D8F7809583
:100CF00090958E0F9F1F08950F931F93CF93DF93AF
:100D0000FB01238121FD03C08FEF9FEF2CC022FF49
:100D100016C046815781248135814217530744F418
:100D2000A081B1819D012F5F3F4F318320838C9340
:100D3000268137812F5F3F4F3783268314C08B0175
:100D4000EC01FB010084F185E02D0995892BE1F68A
:100D5000D80116968D919C911797019617969C93A2
:100D60008E931697CE01DF91CF911F910F91089529
:100D7000FA01AA27283051F1203181F1E8946F93CC
:100D80006E7F6E5F7F4F8F4F9F4FAF4FB1E03ED072
:100D9000B4E03CD0670F781F891F9A1FA11D680F10
:100DA000791F8A1F911DA11D6A0F711D811D911D43
:100DB000A11D20D009F468943F912AE0269F1124B8
:100DC0003019305D3193DEF6CF010895462F47701C
:100DD000405D4193B3E00FD0C9F7F6CF462F4F7077
:100DE000405D4A3318F0495D31FD4052419302D0D5
:100DF000A9F7EACFB4E0A69597958795779567957B
:100E0000BA95C9F700976105710508959B01AC017A
:100E10000A2E06945795479537952795BA95C9F7A1
:100E2000620F731F841F951FA01D08952F923F927C
:100E30004F925F926F927F928F929F92AF92BF92EA
:100E4000CF92DF92EF92FF920F931F93CF93DF9396
:100E5000CDB7DEB7CA1BDB0B0FB6F894DEBF0FBEF3
:100E6000CDBF09942A88398848885F846E847D8440
:100E70008C849B84AA84B984C884DF80EE80FD8042
:100E80000C811B81AA81B981CE0FD11D0FB6F894B8
:0E0E9000DEBF0FBECDBFED010895F894FFCF79
:100E9E0003436F756E742041444330204144433107
:100EAE0000253034752020253034752025303475DA
:0C0EBE00003F065B4F666D7D077F6700FC
:00000001FF
